:0600000000008A013B280C
:080008000900523441344E346A
:1000100044344F344D3420344E3475346D346234AE
:10002000653472342034473465346E346534723448
:100030006134743469346F346E3400344E34653452
:1000400077342034733465346534643420343D347B
:100050000034533465347134753465346E3463342C
:100060006534203463346F346D3470346C346534EB
:100070007434653400348330831681008B12393038
:10008000831290006030F800C92046280D30D3203C
:100090000A30D3200530F0000030F100DF200D30B1
:1000A000D3200A30D320831203130108F000F1019A
:1000B0007008A2007108A3002208F0002308F100D4
:1000C0000330F2000030F300F1207008A200710844
:1000D000A3000D30D3200A30D3201E30F0000030B2
:1000E000F100DF202208F0002308F10098210D30F4
:1000F000D3200A30D3200030A4002408F000F101FE
:100100000A30F2000030F300CA21F201F301C321EA
:100110000319B9282208F0002308F100EC21700827
:10012000A2007108A3002208F0002308F1000A30A1
:10013000F2000030F3003B217008A0007108A1001C
:100140002008F0002108F10098210D30D3200A305A
:10015000D320E530F0000330F100FD212408F00049
:10016000F1010130F2000030F30034217008A400E6
:100170007D280D30D3200A30D3202930F000003004
:10018000F100DF200D30D3200A30D3205328630044
:10019000C728673083160313990018159816831221
:1001A000181698170800831203130C1ED5289900FF
:1001B0000800700FF103F10AF00071040800E62056
:1001C000003803190800D320D920DF2871088A00DD
:1001D000700882007008F60771080318710AF707A3
:1001E0000800F601F701F401F50170087104031D20
:1001F000FA2800347208730403190C29721C0529AB
:10020000EA20031C0529F40DF50D0310F30CF20C84
:100210000310F00DF10DFA287608F0007708F100D0
:1002200000348B13F9007808840079088000F80AFC
:100230008B1708008B13F8037808840000088B17CD
:1002400008000310F20DF30DF40B21290800031030
:10025000F30CF20CF40B272908007208F002730863
:10026000031C730AF10208007208F00773080318F0
:10027000730AF1070800F601F70172087304031905
:10028000FF340130F40073080038031D522972084E
:10029000013A031D52297008F6007108F700F001B9
:1002A000F101003470087104031D57290034F31B59
:1002B0006229F40A740811210130F40021211A2165
:1002C000F400572972081121730811217608F200F1
:1002D0007708F300740811210130F40021211A215C
:1002E000F4007208F6007308F7001A21F3001A21CF
:1002F000F2002D2103187E2934217F297614F4037E
:1003000003190034740811210130F40027211A2147
:10031000F400622900307104031D0800F004080095
:10032000F009F109D928F11F98292D30D320902107
:10033000D001D101D201D301D4010530F500F5037C
:100340000A30F200F3013B21503075078400700839
:10035000303E80007608F0007708F1008A2103190A
:10036000B52975080038031D9F290030F40050306E
:10037000740784000008031DD320F40A7408053AAA
:10038000031DB729080073087102031D08007208D5
:1003900070020800C321031CD029F001F1010800FC
:1003A0000130F000F1010800C321031DCA29D02942
:1003B000C321031DDC29D029C3210319CD2903182A
:1003C000D029CD29C321031DCD29D029F001F10168
:1003D000C321031DD029CD290D30F200F301F120F6
:1003E000EB30F2000C30F30034210800F003700F02
:1003F000F10AF1037008710408000B110B1DFE29AE
:08040000F621031DFD2908008F
:00000001FF
